:020000040000FA
:100000007F28820700340034003401340034003487
:1000100000340A34003400340034643400340034D2
:100020000334E8340034003427341034003401340D
:100030008634A03400340F344234403400349834D1
:1000400096348034820707341134033436340B3449
:10005000173403343A3403341B3400343E340D3443
:1000600020340334423482070A3409340834063415
:100070000534043402340134820753347734653450
:1000800065347034473465346E340034203456346B
:100090006534723431342E34313400345334743492
:1000A000613472347434003445346E346434003452
:1000B000533474346534703400344D3461347234E4
:1000C0006B346534723400345334773465346534BA
:1000D000703469346E3467340034423461346434CB
:1000E000203445346E346434003420344B34483486
:1000F0007A340034433441344C34203400348B019E
:1001000007309F009801831698018C019F0181138D
:10011000FB30850086018312AD01AE01AF01B00155
:10012000B101912291220515AC220E30DE00CC22C5
:100130002930840000309D23D101D5010508D0006D
:1001400003305005CF00501E2E227A230030BB20F2
:100150000430BB20D920031CB2283D233030D222EA
:10016000CE23A8280830BB200C30BB208C23E520F0
:100170007A231D22A628DA002220DE00C7233D2391
:100180005A08013E2220D222CE235A08023E2220C3
:10019000D800030115223D235A08033E2220DD002A
:1001A00017239022A321551AD7283521D22855127A
:1001B00008003608AD003708AE003808AF0039082F
:1001C000B0003D30840010210800D5143E30DD0021
:1001D0005422323028213A300B2142300B213D236A
:1001E0002730D22205113630DD0054222D30DD00BB
:1001F000EE21551A08299122453084001021031858
:1002000005153E213D30840010210318F228F828FE
:10021000D50105150800DD0054225D0828210800DD
:1002200000083002031C2729031D27298403000826
:100230002F02031C2729031D2729840300082E02EF
:10024000031C2729031D2729840300082D02080009
:1002500084002D088000840A2E088000840A2F085C
:100260008000840A300880000800D11839298721CD
:100270003B293E215D21172390220800D7015D080C
:100280008400320880070330D3005721840384039D
:10029000330880070230D3005721840334088007D5
:1002A000840A031C5429800A350880070800570D6A
:1002B000840A8007D30B5729080003305D078400A8
:1002C00002300002031C8629031D79298403623051
:1002D0000002031C8629031D792984035A30000279
:1002E000031C8629031D7929840300300002031CA6
:1002F00086295D08840000308000840A5A3080001E
:10030000840A62308000840A02308000080097214D
:100310003E2103305D078400801F952980018403FE
:100320008001840380018403800197210800B209C1
:10033000B309B409B509B20FA229B30FA229B40FAA
:10034000A229B50A0800D221551AD1290508D000E2
:10035000E32305085006031DA32903305005CE00F2
:100360004F060319A3290310CF0D4E08CF064F08DF
:100370000239D2005106D101CF18C6294E08CF004C
:10038000DC035C18A329DC18A329CF290230D10093
:100390004E08CF00DC0A5C18A329DC18A3294E08FC
:1003A000CF000800D518122A051AEE29851DFA2952
:1003B0002030D6005510DA23051AEA29851DFA29BE
:1003C000D603031DDB29013015220430D600551455
:1003D000D511DB290130D519122A0D2A8519122AC7
:1003E000DA238519F829D518F029051EFA29F029EC
:1003F0005516122A2030D6005510D515DA23051AC5
:100400000C2A85190C2AD603031DFE29FF3015225C
:100410000430D6005514FE29FF305518122A152233
:10042000051ED229D5115510080058070739D800E4
:100430003320D9001D22172308000430D3003530A3
:1004400084005808D7000310D70DD70D5708012096
:1004500080008403D70AD30B262A0800D51436302F
:10046000840004309D233630DD0017238C30582360
:100470003D30D2229022A321051A4E2AB501B401A3
:10048000B3010430D01D8030B200D118482A972122
:100490002930DD003E213630DD003A2A2930840043
:1004A0000301A723D5100800AD01AE01AF01B001D3
:1004B000B1012030D3002908A5002A08A6002B0886
:1004C000A7002C08A8005D0884000310251C822AC0
:1004D0000008AE07031C712AAF0F712AB00F712AF2
:1004E000B10A840A0008AF07031C792AB00F792AE1
:1004F000B10A840A0008B007031C7F2AB10A840AE3
:100500000008B107B10CB00CAF0CAE0CAD0CA80CD0
:10051000A70CA60CA50C5D08D30B642AB10108003A
:1005200054222D3084000008C9000830C800C90CCE
:10053000031C9E2A861506150611A12A861106158A
:100540000611C80B972A840A32300402031C932A2E
:1005500086178613C7230800D723033086000616A4
:10056000D7230612033086000616DA23061203305C
:1005700086000616DA230612023086000616DD23F0
:1005800006122030582308305823013058230630F3
:1005900058230E30582308000030D2220930D222CE
:1005A000CC230800DB003C20FF390319DB2A5C2345
:1005B000DB0A5B08D32A08002030C600A001A10195
:1005C000A201A301A4015D0884000008A500840A1B
:1005D0000008A600840A0008A700840A0008A800F2
:1005E0000310A50DA60DA70DA80D03182514A00D29
:1005F000A10DA20DA30DA40DC603031D002B080021
:10060000203084000C23840A0C23840A0C23840ADF
:100610000C23840A0C23F02A03300007C700C719F3
:10062000800030300007C700C71B80000800DC22B4
:100630000230582320305C23230E35232308352332
:100640002C305C23220E352322083523210E35233E
:100650002E305C2321083523200E35232008352336
:100660003830D2223823C72308000F39303E5C2BA4
:10067000803059045823C72308000130582308004C
:100680008601831608308600831206138616FF3013
:10069000CC0006160608CB00061200000000061665
:1006A00000000612CC030319572BCB19492B080065
:1006B000CA00D40106135F2BCA0054140617402346
:1006C00086018316003086008312861206135418A2
:1006D0000617F03086054A0E0F398604061600000C
:1006E0000612F03086054A080F3986040616000007
:1006F000061208003630DD00840008309D233A30B1
:1007000084000C309D233E30840010309D23423005
:10071000840014309D230800363084000830A7235D
:100720003A3084000C30A7233E3084001030A723D9
:10073000423084001430A7230800F0000430D300B6
:10074000C0238000F00A840AD30BA02B0800F0001D
:100750000430D3000008B123840AF00AD30BAA2B7B
:10076000080083169A0070089B001C1555309D00E8
:10077000AA309D009C149C18BB2B1C1183120800EE
:10078000831670089B001C141A0883120800F130AD
:1007900086055E0886040800D123D123D123D12306
:1007A0000800D423D4230800FF30CC00E52B803090
:1007B000CC00E52B4030CC00E52B2030CC00E52BE5
:1007C0001030CC00E52B0230CC00FF30CD00CD0B3B
:0807D000E72BCC0BE52B080020
:084000005700330043004400A7
:02400E00213F50
:10420000CA0017005C0022008000960098000000A1
:10421000800084001E00000020000B002000000031
:104220006400000000000000D00047001F000000F4
:00000001FF
